:1000000000308A00312800002A30840000080319DB
:1000100018280130A100A001A00B0C28A10B0B286F
:100020004A30A000A00B122800000000800B092815
:10003000003483168510831285140230A90096308F
:10004000AA000420A90B1F2883168510831285108F
:100050000230A9009630AA000420A90B2A281928EA
:10006000452884011F30830507309F000130A5001B
:10007000A601A701A8018316051183120511831695
:10008000051483120518452819286430AA00042095
:1000900083160511831205150130AA00042083166A
:0A00A0000511831205113F286300CB
:02400E00393F38
:00000001FF
